:020000040800F2
:100000006806002065010008050700082B040008A9
:1000100000000000000000000000000000000000E0
:1000200000000000000000000000000009070008B8
:100030000000000000000000070700080B07000890
:1000400077010008770100087701000877010008B0
:1000500077010008770100087701000877010008A0
:100060007701000877010008770100087701000890
:100070007701000877010008770100087701000880
:100080007701000877010008770100087701000870
:100090007701000877010008770100087701000860
:1000A0007701000877010008770100087701000850
:1000B0007701000877010008770100087701000840
:1000C00000F002F800F03EF80CA030C80838241800
:1000D0002D18A246671EAB4654465D46AC4201D180
:1000E00000F030F87E460F3E0FCCB6460126334274
:1000F00000D0FB1AA246AB4633431847C4060000A3
:10010000E4060000103A02D378C878C1FAD8520742
:1001100001D330C830C101D504680C6070470000BD
:100120000023002400250026103A01D378C1FBD813
:10013000520700D330C100D50B6070471FB51FBDFB
:1001400010B510BD00F041F91146FFF7F7FF00F0C0
:1001500017FB00F059F903B4FFF7F2FF03BC00F0FE
:100160005DF900000748804707480047FEE7FEE7C3
:10017000FEE7FEE7FEE7FEE704480549054A064BB1
:10018000704700007D070008C100000868000020DB
:1001900068060020680200206802002001E004C018
:1001A000091F0429FBD28B0701D50280801CC907D7
:1001B00000D00270704700290BD0C30702D0027034
:1001C000401C491E022904D3830702D50280801CEB
:1001D000891EE3E70022EEE70022DFE700220309A1
:1001E0008B4273D3030A8B4258D3030B8B423CD30D
:1001F000030C8B4221D312E003460B437FD4002231
:1002000043088B4274D303098B425FD3030A8B42AA
:1002100044D3030B8B4228D3030C8B420DD3FF2214
:10022000090212BA030C8B4202D31212090265D0E2
:10023000030B8B4219D300E0090AC30B8B4201D395
:10024000CB03C01A5241830B8B4201D38B03C01ADC
:100250005241430B8B4201D34B03C01A5241030B53
:100260008B4201D30B03C01A5241C30A8B4201D304
:10027000CB02C01A5241830A8B4201D38B02C01AAF
:100280005241430A8B4201D34B02C01A5241030A26
:100290008B4201D30B02C01A5241CDD2C3098B420B
:1002A00001D3CB01C01A524183098B4201D38B0188
:1002B000C01A524143098B4201D34B01C01A52412B
:1002C00003098B4201D30B01C01A5241C3088B4270
:1002D00001D3CB00C01A524183088B4201D38B005B
:1002E000C01A524143088B4201D34B00C01A5241FD
:1002F000411A00D201465241104670475DE0CA0FD4
:1003000000D04942031000D34042534000229C4693
:1003100003098B422DD3030A8B4212D3FC2289019D
:1003200012BA030A8B420CD3890192118B4208D373
:10033000890192118B4204D389013AD0921100E0D5
:100340008909C3098B4201D3CB01C01A52418309E9
:100350008B4201D38B01C01A524143098B4201D316
:100360004B01C01A524103098B4201D30B01C01A41
:100370005241C3088B4201D3CB00C01A52418308BB
:100380008B4201D38B00C01A5241D9D243088B4211
:1003900001D34B00C01A5241411A00D201466346B4
:1003A00052415B10104601D34042002B00D5494218
:1003B000704763465B1000D3404201B50020C04641
:1003C000C04602BD704770477047754600F022F87E
:1003D000AE46050069465346C008C000854618B0C1
:1003E00020B5FFF7C9FE60BC00274908B6460026C5
:1003F000C0C5C0C5C0C5C0C5C0C5C0C5C0C5C0C5D5
:10040000403D49008D4670470446C046C0462046E0
:10041000FFF7A1FE004870470400002001491820A2
:10042000ABBEFEE7260002007047FEE708B50449B0
:100430004A6902434A6149690140009108BD0000D0
:100440000010024008B50449CA690243CA61C9697B
:100450000140009108BD000000100240F0B40023EC
:100460000A68002A51D001240A689C402240002AD0
:1004700047D04C68012C01D0022C10D18D68144655
:10048000866864436700E719BE436C432643866071
:10049000CD680C684668A6436C43264346600F69E6
:1004A0001446C668644365006519AC46AE432546EC
:1004B0007D432E43C6604D68022D1BD1FF2A0CD808
:1004C0004F691646056A2246724372431601B61AF0
:1004D000B5437A43154305620CE04E69150A2A4676
:1004E0006A436A436A431501476AAD1AAF437243D0
:1004F000174347624A6805686646B5435443254337
:1005000005605B1C0A68DA40ADD1F0BC0020704782
:1005100010B57D21C900FFF761FE0449401E486106
:10052000002088610520086110BD000000E000E0A7
:1005300030B4012203685B06DB0FD402002B2DD1FF
:100540004B680A680D691A43CB682B431A434B6901
:100550001A438B691A43CB691A430B6A1A4303681F
:10056000114D2B401A4302604268104B1A404B69F0
:100570001B0C1A438B681A4342608A68A24204D259
:10058000630042689A431A43426001230A6A5B038C
:100590009A4202D1898C89B201610022C169A143CA
:1005A000C16130BC104670474000FFFFFBF0FFFF09
:1005B00001490860704700000000002070B586B057
:1005C00018216846FFF708FE0120C004FFF72EFF40
:1005D00001208005FFF72AFF01208004FFF726FF96
:1005E00001204004FFF722FF01201A4D8002A8627B
:1005F0000821A9622021A9624021A96200240126C4
:100600000090029403946946019604942846FFF7EB
:1006100025FF0820009002940394694601960494F3
:100620002846FFF71BFF20200090029403946946A0
:10063000019604942846FFF711FF40200090029491
:1006400003946946019604942846FFF707FF06B015
:1006500070BD000000040048F0B591B0282106A844
:10066000FFF7BAFD18216846FFF7B6FD0127BF0363
:100670003846FFF7E7FE3801FFF7D8FE0024781070
:1006800002250326039404946A46059461C26946D0
:100690001A48FFF7E3FE009703940494694617484D
:1006A000029601950594FFF7D9FEA80303940494DC
:1006B0006A46059461C269461048FFF7CFFEFF20E5
:1006C00005300790300208900694099428020A9495
:1006D0000C940D940E940B900720094C0F9006A9D2
:1006E0002046FFF725FF606810218843606060683E
:1006F00008210843606011B0F0BD0000000400480C
:1007000000380040FEE770477047704710B5184842
:1007100001684908490001600168C907C90FFBD198
:100720001448016801221143016001688907C90F5B
:10073000FBD00168F8229143802211430160416897
:10074000F0229143416041680722120291434160C7
:1007500041688908890041600C2241681142FCD13E
:10076000054C2046FFF7D4FE2046FFF721FF10BDC1
:10077000002002400010024000127A007047000082
:1007800008B50D48012182690A43826180690840E9
:1007900000900807FFF756FE0848C16903220902C6
:1007A000090A92071143C161FFF7B0FFFFF706FF87
:1007B000FFF752FFFEE700000010024004ED00E0EA
:1007C000E007000800000020040000000401000809
:1007D000E40700080400002064060000200100086F
:0407E00000127A0089
:04000005080000C12E
:00000001FF
